:100000000C941E060C94D2270C94FF270C944606E1
:100010000C9446060C9446060C9446060C94460630
:100020000C9446060C9446060C94EF120C9446066B
:100030000C9446060C9446060C9446060C94460610
:100040000C942C280C9446060C941A2C0C945D2CC1
:100050000C9446060C9446060C9446060C944606F0
:100060000C9446060C9446065318B5189418971825
:100070009A189D18A018A318A618B518AF18E71954
:10008000E919E919E719E919E919E919E919E91962
:10009000E919E919E919E919E919E919E919E91950
:1000A0006D19E919E919E919E919E919DE18E919C8
:1000B000E919E919E919E919E919E919E919E91930
:1000C000E919E919E919E919E919E9197919791900
:1000D0007919791979197919791979197919E91920
:1000E000E919E919E919E919E919DE1878197819EE
:1000F00078197819E91986198C19921998199E1985
:10010000A419AA19B019BA19C419CE19D8191F19E6
:10011000E118E919E919E919E9196D19E919E91954
:10012000E919E919E919E919E919E91977197719A3
:1001300077197719E91986198C19921998199E1946
:10014000A419AA19B019BA19C419CE19D8191F19A6
:10015000E118E919E919E919E9196D191C1A1C1AAC
:100160001C1A1C1A1C1A1C1A1C1A1C1A1C1A1C1ADF
:100170001C1A1C1A1C1A331B331B331B331B331B57
:10018000331B611A6B1A751A7F1ADD1AE71AF61AF1
:10019000071B8F1CA41CB01CB91CC81CED1CF61C32
:1001A0003F1D081D512057205D206420722094209F
:1001B000B220456E746572206D656E752E2E2E0010
:1001C000546F67676C6564206D6963726F50504D42
:1001D00000546F67676C656420696E76657274653C
:1001E000642050504D2100546F67676C6564205443
:1001F00058206D7574696E672100546F67676C6570
:10020000642074656C656D65747279210050726F3D
:10021000746F636F6C206572726F72207769746897
:100220002052580054696D656F7574207768656E4B
:1002300020636F6E6E656374696E6720746F205201
:100240005800507265737320616E79206B65792058
:10025000746F2063616E63656C00436F6E6E6563DF
:1002600074696E6720746F2052582C20706F776508
:100270007220757020746865205258202877697440
:10028000682062696E6420706C7567206966206EF4
:100290006F74207573696E6720616C776179732064
:1002A00062696E642900546F67676C656420276912
:1002B0006D6D656469617465206F75747075742700
:1002C00000546F67676C65642027736C61766520E6
:1002D0006D6F64652700546F67676C6564202761E4
:1002E0006C776179732062696E642700546F676769
:1002F0006C65642050504D206368616E6E656C20A3
:100300006C696D69740053657420525353492069B8
:100310006E6A656374696F6E206368616E6E656C8A
:100320002028303D3D64697361626C652900536526
:10033000742050504D206D696E696D756D20737914
:100340006E630053657420626561636F6E20696E31
:1003500074657276616C0053657420626561636FC9
:100360006E2064656C617900536574206265616319
:100370006F6E206672657175656E637920696E2097
:10038000487A3A20303D64697361626C652C205074
:10039000783D504D52206368616E6E656C20782CFC
:1003A0002046783D465253206368616E6E656C202E
:1003B00078005365742050574D2073746F7020641B
:1003C000656C61792028302064697361626C6564B2
:1003D0002C20312D323535203D3D20302E317320FB
:1003E0002D2035306D696E29005365742050504DB5
:1003F0002073746F702064656C61792028302064EC
:10040000697361626C65642C20312D323535203D75
:100410003D20302E3173202D2035306D696E29003E
:10042000536574206661696C736166652064656CF0
:1004300061792028302064697361626C65642C20C6
:10044000312D323535203D3D20302E3173202D2089
:1004500035306D696E29002A2A2A2A2A2A2A2A2A50
:100460002A2A2A2A2A2A2A2A2A2A2A2A2A2A2A2AEC
:100470002A2A2A2A0052582041636B6564202D20C5
:1004800072657665727420737563636573736675E0
:100490006C21002A2A2A2A2A2A2A2A2A2A2A2A2AAD
:1004A0002A2A2A2A2A2A2A2A2A2A2A2A2A2A2A2AAC
:1004B000002A2A2A2A2A2A2A2A2A2A2A2A2A2A2AC6
:1004C0002A2A2A2A2A2A2A2A2A2A2A2A2A2A00528E
:1004D000582041636B6564202D20757064617465DC
:1004E000207375636365737366756C21002A2A2A0D
:1004F0002A2A2A2A2A2A2A2A2A2A2A2A2A2A2A2A5C
:100500002A2A2A2A2A2A2A2A2A2A0056616C696457
:100510002063686F69636573206172653A205B319F
:100520005D2D5B31365D20286368616E6E656C20E1
:10053000312D31362900536574206F7574707574D0
:1005400020666F7220706F727420005B585D2061AE
:10055000626F7274206368616E67657320616E6498
:10056000206578697420525820636F6E6669670051
:100570005B535D20736176652073657474696E6783
:100580007320746F205258005B525D20726576654F
:1005900072742052582073657474696E6773207486
:1005A0006F2064656661756C747300557365206EA9
:1005B000756D62657273205B312D445D20746F2010
:1005C0006564697420706F727473205B452D515D92
:1005D00020666F722073657474696E677300202DD6
:1005E00020726563656976657220636F6E66696700
:1005F000757261746F722C20727820737720000AF4
:100600000A6F70656E4C52536E67200053657420FC
:1006100073657269616C2062617564726174653AB8
:10062000200056616C69642063686F696365733A82
:100630002031202D20342B34202F2032202D203823
:10064000202F2033202D20382B34202F2034202D14
:10065000203132202F2035202D2031322B34202FF5
:100660002036202D20313600536574204368616E9A
:100670006E656C20636F6E6669673A20005365741F
:100680002044617461726174652028302D32293AEA
:10069000200053657420486F70206368616E6E653A
:1006A0006C7320286D61782032342C207365706162
:1006B000726174656420627920636F6D6D61732966
:1006C0002076616C69642076616C75657320312DCC
:1006D0003235353A2000536574206368616E6E656B
:1006E0006C2073706163696E6720287831306B48C5
:1006F0007A293A200053657420524620706F77653E
:10070000722028302D37293A200053657420524634
:10071000206D6167696320286865782920652E67E8
:100720002E20307844454144463030443A2000532E
:1007300065742062617365206672657175656E63AC
:10074000792028696E20487A293A20005B5A5D207A
:10075000656E746572207265636569766572206383
:100760006F6E66696775726174696F6E2075746902
:100770006C79005B465D20646973706C61792061FF
:10078000637475616C206672657175656E63696509
:10079000732075736564005B525D2063616C6375E3
:1007A0006C6174652072616E646F6D206B65792079
:1007B000616E6420686F70206C697374005B495DC2
:1007C000207265696E697469616C697A6520736508
:1007D0007474696E677320746F20736B65746368DB
:1007E0002064656661756C7473005B585D2072658A
:1007F00076657274206368616E67657320616E64EC
:100800002065786974206D656E75005B535D20739B
:100810006176652073657474696E677320746F20E8
:10082000454550524F4D20616E64206578697420B3
:100830006D656E7500557365206E756D62657273BA
:10084000205B302D395D20746F20656469742070E1
:100850006172616D657465727300202D2053797328
:1008600074656D20636F6E66696775726174696F18
:100870006E000A0A6F70656E4C52536E672000510D
:1008800029204F7574707574206265666F726520DB
:100890006C696E6B20283D465329203A2000502970
:1008A00020536C617665206D6F64652028657870D3
:1008B0006572696D656E74616C293A20004F29205C
:1008C00054696D65642042494E44206174207374FC
:1008D000617274757020203A20004E292050504DCE
:1008E000206F7574707574206C696D69746564200F
:1008F000202020203A200044495341424C454400E6
:100900004D292050504D205253534920746F20637D
:1009100068616E6E656C202020203A20004C2920F2
:1009200050504D206D696E696D756D2073796E63E1
:10093000202875732920203A200044495341424C15
:100940004544004B29204661696C736166652062ED
:100950006561636F6E20696E74762E2028312D32AA
:10096000353573293A20004A29204661696C736144
:10097000666520626561636F6E2064656C617920D5
:1009800028302D323535203D3E20313073202D204A
:100990003135306D696E293A200049292046616958
:1009A0006C7361666520626561636F6E206672714B
:1009B0002E203A200048292050574D2073746F7024
:1009C0002064656C6179202020202020203A2000BE
:1009D00047292050504D2073746F702064656C61FE
:1009E00079202020202020203A200046292046611E
:1009F000696C736166652064656C617920202020D4
:100A00002020203A200050574D206368616E6E65AB
:100A10006C200066756E6374696F6E3A2000292041
:100A2000706F72742000506F776572546F776572C3
:100A300000445446205548462033322D62697420C4
:100A400031306368004F70656E4C52536E67525878
:100A5000206D696E6920342F36636800466C7974A6
:100A6000726F6E2F4F72616E6765525820554846FF
:100A70002038636800525820747970653A20004429
:100A8000697361626C656400487A00203D3D200016
:100A900043616C63756C61746564207061636B6540
:100AA0007420696E74657276616C3A200042292068
:100AB0004D6963726F202868616C66292050504D23
:100AC000202020203A00412920496E766572746505
:100AD000642050504D20696E20202020203A0030A4
:100AE00029204D7574652062757A7A657220286DAB
:100AF0006F73746C79293A003929205365726961E2
:100B00006C2062617564726174653A00736D617224
:100B100074506F7274004672536B79005472616E38
:100B200073706172656E740044697361626C6564B0
:100B30000038292054656C656D657472793A2020FF
:100B40002020202020003729204368616E6E656CCC
:100B500020636F6E6669673A202000362920446161
:100B60007461726174652028302D32293A2020206A
:100B700000352920486F70206368616E6E656C7364
:100B80003A2020202020003429204368616E6E65C1
:100B90006C2073706163696E673A202000332920EE
:100BA000524620706F7765722028302D37293A2001
:100BB0002020003229205246206D616769633A2067
:100BC0002020202020202020003129204261736530
:100BD000206672657175656E63793A202020000089
:100BE00000000700020100000304060000000000EE
:100BF00000000001020408102040800102040810D7
:100C00002001020408102004040404040404040263
:100C10000202020202030303030303000000002395
:100C2000002600290000000000250028002B0000FD
:100C3000000000240027002A00004B2D11241FBEB5
:100C4000CFEFD8E0DEBFCDBF13E0A0E0B1E0E4EA33
:100C5000F0E602C005900D92A83CB107D9F716E066
:100C6000A8ECB3E001C01D92AE38B107E1F71CE07B
:100C7000CCE3DCE004C02297FE010E94542ECA336C
:100C8000D107C9F70E94872D0C9450300C940000B6
:100C900080917305813019F482E08093730580910F
:100CA0007305833019F484E0809373050895A89543
:100CB0000895DC01ED91FC910190F081E02D099502
:100CC00008952091740530917505382748E0C901D1
:100CD000880F991F37FF06C09C0151E2252750E17C
:100CE000352701C09C01415091F730937505209341
:100CF0007405089588E38093760580E092ECA1E086
:100D0000B0E08093770590937805A0937905B09330
:100D10007A0587E08093830580EC92E9ADEEB9E136
:100D200080937B0590937C05A0937D05B0937E0511
:100D300085E0809384058DEE9EEFADEABEED809355
:100D40007F0590938005A0938105B0938205E5E827
:100D5000F5E080E090E0863028F4DC01AE54BC4F32
:100D60002C9101C020E0219301968831910599F7DB
:100D700082E080939D058AE080939E05089580EC33
:100D800091EDA8E9BBE18093BB059093BC05A093CE
:100D9000BD05B093BE0580E090E0A0E0B0E5809393
:100DA000BF059093C005A093C105B093C205E3ECC5
:100DB000F5E080E081938F5F8031E1F70895A0E056
:100DC000B0E0E5EEF6E00C941D2ED82F0E948228AC
:100DD0006115710581059105C9F30E94C02E10921D
:100DE0007F05109280051092810510928205C4E063
:100DF000812C912C54018A94C0907F05D09080055D
:100E0000E0908105F0908205FE2CED2CDC2CCC24AA
:100E10000E94BB2EA50194010E94FC2D6C0D7D1D2E
:100E20008E1D9F1D60937F057093800580938105C3
:100E300090938205C15001F7DD2309F450C005E805
:100E400015E0E801A12CB12C62E3C62ED12CE12CD7
:100E5000F12C8881882309F442C0B39419F40E94CC
:100E60007A063DC00E94BB2EA70196010E94FC2D70
:100E7000E1E0E60FA5E8B5E08A2F801B8A1520F493
:100E80008D918E13F9CFE9CF2091840530E0A0E158
:100E9000B7E20E94942D9B01AC01AE2FB0E00E94FE
:100EA000A32D40907B0550907C0560907D0570904F
:100EB0007E05640D751D861D971D4090BB055090E5
:100EC000BC056090BD057090BE05461657066806C5
:100ED000790618F2E993A39488E1A812BACFCDB7A6
:100EE000DEB7E0E10C94392E8436910520F4BC0184
:100EF00080E090E017C09C018E3B910528F42A55B4
:100F00003109AAE0B0E00CC0823D910528F4245BD1
:100F10003109A4E6B0E004C02D5C3109A8E5B2E0D7
:100F20000E94942DA4E6B0E09B01AC010E94A32D89
:100F3000089590E08C599F4F0E947407089561E0D6
:100F40008FE00E942F2960E08FE00E9468290895B9
:100F5000892B11F061E001C060E08FE00E946829F8
:100F6000089560E08CE00E942F2961E08BE00E94F0
:100F70002F2961E08DE00E942F2960E082E00E942D
:100F80002F2961E084E00E942F29089542E050E07B
:100F900068E476E080E00E94B2270895E3E0F0E0A4
:100FA00089E080935700E491E67081E0E63009F033
:100FB00080E00895CF93DF93C82F0E94CE07882347
:100FC00081F0DFB781E080937205F8940E945706A4
:100FD00088E180936000C0936000C1110E945706B1
:100FE000DFBFDF91CF9108958F929F92AF92BF9212
:100FF000CF92DF92EF92FF92CF93FC01C0A5EC2F2E
:10100000E770F0E0E658FC4FA081B0E0C7FF03C0F6
:1010100024E130E002C02FE030E0FC0197A183E141
:10102000989FF0011124E25CFE4F80809180A280A5
:10103000B380A20FB31F20E43FE14DE750E00E94D0
:10104000AE2DA50194010E94DA2D8C2F887149F4F0
:1010500069017A01E0EDCE0EE7E0DE1EE11CF11C35
:101060001BC0C7FF05C060E47AE88CE29EE004C0C4
:1010700060E07EEE8AEB9BE069017A01F8EBCF0E2F
:10108000FBE0DF1EE11CF11CA50194010E94DA2D9A
:10109000C20ED31EE41EF51EC701B60169517C4F76
:1010A0008F4F9F4F28EE33E040E050E00E94DA2D52
:1010B000A8EEB3E00E94A32DCF91FF90EF90DF90B8
:1010C000CF90BF90AF909F908F9008958F3F9105E4
:1010D00051F048F0811522E0920738F081159340D5
:1010E00030F482E0089580E0089581E0089583E07F
:1010F0000895A0E0B0E0EFE7F8E00C94262EEB01B5
:101100008A01B82FB695A0E028813981F8012083A3
:101110002A813B8121832C813D8122832E813F8145
:101120002383688179814A815B812C813D81EE81B5
:10113000FF819F2F9295990F990F907C272F2370F5
:10114000922B252F2370220F220F922B232F2370F7
:101150002295207F922BF80194830B5F1F4F2896D6
:10116000AF5FBA1788F680FF24C0888199810E94FA
:101170006608D82E8A819B810E946608E82E8C81A1
:101180009D810E946608F82E8E819F810E946608CC
:10119000F0E4DF9EA001112490E1E99E900111246A
:1011A000242B282BE4E0FE9EB0011124262BF8010D
:1011B0002083CDB7DEB7E7E00C94422E803223E0E7
:1011C000920708F1883E23E0920740F48F51934044
:1011D000E4E096958795EA95E1F70895803D27E04C
:1011E000920718F48C5D93400895883928E092079F
:1011F00068F4885C974074E0969587957A95E1F756
:101200008D509C4F089580E090E008958FEF93E01B
:1012100008958C30910540F4A4E0880F991FAA9599
:10122000E1F7885D9C4F0895843F23E0920718F40E
:1012300084529C4F0895811524E0920740F486570C
:10124000934FF4E0880F991FFA95E1F7089580E92C
:1012500098E008959C013695279525753575821B74
:10126000930B9C0123733373969587959695879579
:1012700083739373820F931F9C0154E036952795D7
:101280005A95E1F7280F391F2F703F7041E051E068
:10129000249FC001259F900D349F900D1124892F0C
:1012A00008952D98882319F000002B9A02C00000A1
:1012B0002B9800002D9A000008952D9A000083B10C
:1012C0002D980000829581700895CF93DF93D82FD9
:1012D0005C9A2D985C98C8E08D2F80780E94510907
:1012E000DD0FC150C9F72D98DF91CF9108958F7709
:1012F0000E9465090895CF93DF93D82FC8E08D2F02
:1013000080780E945109DD0FC150C9F72D98DF91F7
:10131000CF910895CF93DF932D98C8E080E0D82F28
:10132000DD0F0E945D098D0FC150C9F7DF91CF918C
:1013300008950E9477090E948A095C9A0895A1E0A5
:10134000B0E0E5EAF9E00C942B2E806869830E94F6
:1013500065096981862F0E947B095C9A2196E2E0EB
:101360000C94472ECF93C0917F05C827E82FF0E05B
:10137000EA58FA4F678589E70E949F096C2F8DE331
:101380000E949F096C2F82E40E949F09CF910895CB
:1013900086E20E9499090895CF93DF93EC016C8156
:1013A0008CE10E949F096D818DE10E949F096E81F1
:1013B0008EE10E949F096F8180E20E949F096885EB
:1013C00081E20E949F09698582E20E949F096A85E5
:1013D00083E20E949F096B8584E20E949F096C85CD
:1013E00085E20E949F096D858AE20E949F096E85B1
:1013F0008EE60E949F096F858FE60E949F0968898B
:1014000080E70E949F09698981E70E949F096A8994
:1014100082E70E949F09DF91CF910895CF92DF92DA
:10142000EF92FF92CF93DF936B017C01C11488E3AD
:10143000D8068CE9E8068CE1F80628F5C701B60164
:1014400020E836E948E950E00E94DA2DE901689782
:1014500060E879E687E69FEF0E94B62D6C0D7D1D52
:101460008E1D9F1DF2E0660F771F881F991FFA954A
:10147000D1F721E732E040E050E00E94DA2DF22E71
:10148000E32E80E421C0C701B60120E03DE241E344
:1014900051E00E94DA2DE901689760E073ED8EEC6F
:1014A0009EEF0E94B62D6C0D7D1D8E1D9F1D660F3B
:1014B000771F881F991F21E732E040E050E00E942B
:1014C000DA2DF22EE32E80E66C2F6F71680F85E720
:1014D0000E949F096E2D86E70E949F096F2D87E766
:1014E0000E949F09DF91CF91FF90EF90DF90CF9006
:1014F0000895682F8DE60E949F0908958F929F920C
:10150000AF92BF92CF92DF92EF92FF92CF93DF9391
:10151000D82F83E00E9499098093710584E00E948E
:1015200099098093700560E086E00E949F0961E060
:1015300087E00E949F096FE789E00E949F0965E0AC
:101540008AE00E949F0962E18BE00E949F0965E1A9
:101550008CE00E949F096DEF8DE00E949F0960E082
:101560008EE00E949F09DD2319F08BE291E008C014
:1015700020919D0533E1239FC0011124825C9E4F81
:101580000E94CC096CE880E30E949F096FE082E32F
:101590000E949F0962E483E30E949F0980919E0557
:1015A00087FF02C064E101C06AE084E30E949F09F2
:1015B0006AE285E30E949F096DE286E30E949F092B
:1015C00064ED87E30E949F0960E088E30E949F0921
:1015D00060E089E30E949F09D11109C0C0907F0596
:1015E000D0908005E0908105F090820507C0C5E9A4
:1015F000CC2EC1ECDC2EED2CCEEDFC2ECAE38F2CD4
:101600009924AA24BB24682D8C2F0E949F09682D41
:1016100085E08C0F0E949F09FE2CED2CDC2CCC2445
:10162000CF5FCE3361F76FEF83E40E949F096FEFC6
:1016300084E40E949F096FEF85E40E949F096FEF89
:1016400086E40E949F09DD2311F066E002C06091EC
:1016500083058DE60E949F0960E089E70E949F094B
:10166000609184058AE70E949F0960E083E70E94F9
:101670009F0960E084E70E949F09D11109C0609131
:101680007B0570917C0580917D0590917E0504C05D
:1016900060EC72E98DEE99E10E940E0ADF91CF9124
:1016A000FF90EF90DF90CF90BF90AF909F908F9082
:1016B000089561E087E00E949F0964E28EE70E943E
:1016C0009F0963E088E00E949F0960E088E00E9433
:1016D0009F0965E087E00E949F0962E085E00E9423
:1016E0009F0983E00E9499098093710584E00E941C
:1016F000990980937005089583E00E949909809369
:10170000710584E00E9499098093700561E087E08B
:101710000E949F096AE070E080E090E00E94A528A6
:101720000E94590B00000895CF92DF92FF920F9311
:101730001F93CF93DF931F92CDB7DEB7082F162FDD
:101740008EE399830E949F09F02EC02E9981D92E95
:101750008C2D8F19811738F4F60161916F018FE795
:101760000E949F09F5CF64E085E00E949F0983E015
:101770000E9499098093710584E00E9499098093E1
:1017800070050E94822860936C0570936D058093AC
:101790006E0590936F0569E087E00E949F0981E0E4
:1017A000809373050F90DF91CF911F910F91FF9060
:1017B000DF90CF9008950F931F930E94940B809118
:1017C0007305813099F40E94822800916C05109174
:1017D0006D0520916E0530916F05601B710B820BBA
:1017E000930B603A76488140910548F380917305E8
:1017F000813031F46EE971E082EE95E00E946E2A4C
:101800001F910F9108950F931F938091730582305C
:1018100021F41092730581E020C08091730581301E
:10182000D9F40E94822800916C0510916D052091D9
:101830006E0530916F05601B710B820B930B613A43
:1018400076488140910540F061E087E00E949F0961
:101850001092730582E001C080E01F910F910895FE
:10186000CF93DF93EC014AE050E06D2F70E082EE01
:1018700095E00E943C2B6EE282EE95E00E94402AA9
:10188000BE0184E0769567958A95E1F76F707727BA
:101890004AE050E082EE95E00E943C2B6EE282EE40
:1018A00095E00E94402ABE016F7077274AE050E021
:1018B00082EE95E00E943C2BDF91CF910895D82FC6
:1018C000C0E0CD1790F45E9A409A64E670E080E044
:1018D00090E00E94A5285E98409864E670E080E061
:1018E00090E00E94A528CF5FECCF6CE271E080E031
:1018F00090E00E94A528E4CF0F931F93CF93DF932E
:10190000EC01062F15E0115051F0CE010E94373046
:10191000081741F0602FCE010E943F30F4CF82E0E3
:101920000E945F0CDF91CF911F910F910895A0E06D
:10193000B0E0EDE9FCE00C941D2E482E562EC0E0E0
:10194000D0E0612C712CE12CF12C00E010E0411072
:101950000CC06090D40586E4689E3001112459E1E2
:10196000E52EF12C0AEB15E01EC091E049120FC0E4
:101970006090D405E6E46E9E30011124FBE16F0E09
:10198000711C49E2E42EF12C06E715E00CC082E060
:10199000481209C028E1622E77247394EE24E39460
:1019A000F12C03ED15E043018C0E9D1E1092750580
:1019B000109274053401A62CA818B12CC30101960D
:1019C0006C01AE14BF04A8F4A00EB11E511006C0E5
:1019D000C3010E943730F501808305C0F5016081A5
:1019E000C3010E947C0CF50180810E9461063601D2
:1019F000E2CFC301511018C0C3010E943730B82E86
:101A0000C6010E9437302B2D30E0322F2227282BA1
:101A100080917405909175058217930779F4C0E061
:101A2000D0E05524539493CF3601609175050E9400
:101A30007C0C60917405C6010E947C0CC05EDE4F78
:101A4000C13E92E0D90708F482CF852DCDB7DEB72D
:101A5000E0E10C94392E61E082E00E94970C089539
:101A600060E082E00E94970C8091D305853020F0E1
:101A70001092D3050E942B0D8091D3058093D4053D
:101A8000089561E080E00E94970C61E081E00E948F
:101A9000970C089560E080E00E94970C882351F035
:101AA00060E081E00E94970C882321F08091760508
:101AB000883349F00E94BF060E947A0681E00E94A6
:101AC000DF060E94410D0895882319F06AEA71E04B
:101AD00002C06EEA71E082EE95E00E946E2A0895DF
:101AE000FF920F931F93CF93DF9369EC7BE082EE1D
:101AF00095E00E941A2A40917B0550917C056091E7
:101B00007D0570917E052AE030E082EE95E00E942E
:101B1000432B63EB7BE082EE95E00E941A2A409112
:101B20007F0550918005609181057091820520E1CB
:101B300030E082EE95E00E94432B6DE97BE082EE7F
:101B400095E00E941A2A4AE050E06091830582EEF7
:101B500095E00E946B2B67E87BE082EE95E00E94A7
:101B60001A2A4AE050E06091840582EE95E00E94D6
:101B70006B2B61E77BE082EE95E00E941A2AC5E8B4
:101B8000D5E0F12C8E0188818823A9F0FF2031F067
:101B900061EB71E082EE95E00E943D2A21964AE0D9
:101BA00050E0F801608182EE95E00E94342BF394BE
:101BB000F8E1FF12E7CF82EE95E00E94482A6BE53C
:101BC0007BE082EE95E00E941A2A4AE050E06091A4
:101BD0009D0582EE95E00E946B2B66E47BE082EE31
:101BE00095E00E941A2AE0919E05E770F0E0EE0F62
:101BF000FF1FEE57FC4F6081718182EE95E00E94DD
:101C00006E2A61E37BE082EE95E00E941A2A8091C1
:101C10009E058871883069F028F4811113C068E24C
:101C20007BE00CC0803141F0883161F46CE07BE0F6
:101C300005C06CE17BE002C066E17BE082EE95E0EE
:101C40000E945C2A68EF7AE082EE95E00E941A2AF0
:101C500040917705509178056091790570917A05EA
:101C60002AE030E082EE95E00E94432B6FED7AE0AF
:101C700082EE95E00E941A2A8091BF0580710E9431
:101C8000640D66EC7AE082EE95E00E941A2A80915B
:101C9000BF0580740E94640D6DEA7AE082EE95E0E3
:101CA0000E941A2A8091BF0580720E94640D60E92B
:101CB0007AE082EE95E00E941A2A86E795E00E947B
:101CC000F407AB01BC012AE030E082EE95E00E940F
:101CD000252B6BE87AE082EE95E00E941A2A86E7CF
:101CE00095E00E94F4079B01AC0160E472E48FE090
:101CF00090E00E94DA2DBA01A9012AE030E082EEDC
:101D000095E00E94252B68E87AE082EE95E00E943B
:101D10005C2ACDB7DEB7E5E00C94442E8F929F92FB
:101D2000AF92BF92CF92DF92EF92FF92811107C0E4
:101D30006FE77AE082EE95E00E945C2A2FC090E087
:101D40000E94740724E630E040E050E00E94DA2D63
:101D5000CA01B9012AE030E040E050E00E94DA2DEB
:101D600049015A016B017C012AE030E0B501A40170
:101D700082EE95E00E94252B6EE282EE95E00E94B5
:101D8000402A2AE030E0B701A60182EE95E00E94E9
:101D9000252B63E782EE95E00E94802AFF90EF906A
:101DA000DF90CF90BF90AF909F908F9008951F933A
:101DB000CF93DF9365E77AE082EE95E00E941A2ADE
:101DC00080919F05813041F46CE57AE082EE95E0E8
:101DD0000E945C2A10E050C0823019F465E47AE079
:101DE000F5CF843019F461E37AE0F0CF853091F7D4
:101DF00066E27AE0EBCFC12FD0E0C930D1050CF418
:101E000041C068E3610F82EE95E00E94402A6EE1D6
:101E10007AE082EE95E00E941A2ABE016F5F7F4F42
:101E20004AE050E082EE95E00E94042B63E17AE004
:101E300082EE95E00E941A2AC156DA4FE981E0321B
:101E400018F566E07AE082EE95E00E941A2A898110
:101E5000803130F06DE673E082EE95E00E943D2A1D
:101E600069816F7070E06F5F7F4F4AE050E082EEF3
:101E700095E00E940D2B1F5F80914805181708F40C
:101E8000BACF0FC061E3BECFEF70F0E0EE0FFF1FDF
:101E9000EE56FC4F6081718182EE95E00E946E2AC1
:101EA000EACF6BEE79E082EE95E00E941A2A8091EB
:101EB000B7050E948E0E60ED79E082EE95E00E94FB
:101EC0001A2A8091B8050E948E0E65EB79E082EEA9
:101ED00095E00E941A2A8091B9050E948E0E6AE947
:101EE00079E082EE95E00E941A2A4091AF05509168
:101EF000B0056091B1057091B205411551056105BC
:101F0000710539F12AE030E082EE95E00E94432B22
:101F100067E679E082EE95E00E941A2A8091B30587
:101F20000E949907AB01BC012AE030E082EE95E007
:101F30000E94432B63E479E082EE95E00E941A2A26
:101F40004AE050E06091B40582EE95E00E946B2B70
:101F500006C06AE379E082EE95E00E945C2A6DE1BA
:101F600079E082EE95E00E941A2A6091B5057091A1
:101F7000B6054AE050E082EE95E00E94552B60E005
:101F800079E082EE95E00E941A2A6091AE056034F5
:101F900050F470E06F5F7F4F4AE050E082EE95E0D2
:101FA0000E940D2B06C067EF78E082EE95E00E945C
:101FB0005C2A6AED78E082EE95E00E941A2A809110
:101FC000AD0580FF03C063EB71E002C067EB71E019
:101FD00082EE95E00E946E2A6DEB78E082EE95E04D
:101FE0000E941A2A8091AD0582700E94640D6EE9EC
:101FF00078E082EE95E00E941A2A8091AD05847007
:102000000E94640D6FE778E082EE95E00E941A2A44
:102010008091AD0588700E94640DDF91CF911F9172
:1020200008950F931F93CF93DF93209145052F3F82
:10203000A9F56FEF75E082EE95E00E941A2A83E819
:1020400093E00E94300C6EED75E082EE95E00E9408
:102050001A2A80914605909147050E94300C6BEA40
:1020600075E082EE95E00E945C2A68E875E082EEF9
:1020700095E00E945C2A60E775E082EE95E00E94A0
:102080005C2A6BE475E082EE95E00E945C2A82EEA9
:1020900095E00E94482A0E94D70E68C012160CF0E4
:1020A00065C0332727FD30958091480590E0821761
:1020B00093070CF45BC066E375E082EE95E00E9446
:1020C0001A2A60914505772767FD70954AE050E030
:1020D00082EE95E00E940D2B6BE075E082EE95E0BC
:1020E0000E941A2A10E008E2809149051817D0F5DD
:1020F000C12FD0E0CC0FDD1FC65BDA4F288130E066
:1021000080914505992787FD9095019728173907F4
:1021100039F56BEB71E082EE95E00E943D2A4AE0D2
:1021200050E0602F82EE95E00E94342B6FEB71E05F
:1021300082EE95E00E943D2AE981EF70F0E0EE0F1B
:10214000FF1FEE56FC4F6081718182EE95E00E9488
:102150003D2A63EC71E082EE95E00E943D2A0F5F1C
:102160001F5FC2CF82EE95E00E94482ADF91CF9197
:102170001F910F910895FF920F931F93CF93DF93B9
:10218000C5E8D5E0F12C8E0188818823D1F165EC7A
:1021900071E082EE95E00E943D2A4AE050E06F2D0A
:1021A00082EE95E00E94342B62ED71E082EE95E0C4
:1021B0000E943D2A2196F801208130E0A0E1B7E29B
:1021C0000E94942D9B01AC01A0918405B0E00E9477
:1021D000A32DAB01BC0180917B0590917C05A09162
:1021E0007D05B0917E05480F591F6A1F7B1F2AE0AD
:1021F00030E082EE95E00E94432BF394F8E1FF1269
:10220000C2CFCDB7DEB7E5E00C94442E1092DF04C8
:1022100085E6E0EEF4E0DF011D928A95E9F7089586
:10222000CF93C82F8F3719F0883009F045C0E0915F
:10223000DF04EE23D9F1E150E093DF04F0E0E05257
:10224000FB4F10826DE070E082EE95E00E9459062F
:10225000C0E08091DF04C81760F4EC2FF0E0E0529A
:10226000FB4F608170E082EE95E00E945906CF5FDF
:10227000F0CF60E270E082EE95E00E9459066DE0DA
:1022800070E082EE95E00E945906C0E08091DF0484
:10229000C81778F5EC2FF0E0E052FB4F608170E05A
:1022A00082EE95E00E945906CF5FF0CF67E082EEA4
:1022B00095E00E94402A1DC08B3119F40E9406113E
:1022C0001AC08D30C1F08A30B1F08091DF048436BD
:1022D00068F76C2F70E082EE95E00E945906E0915D
:1022E000DF0481E08E0F8093DF04F0E0E052FB4FCB
:1022F000C08380E001C081E0CF910895CF93C82FC3
:102300000E9482286093C8047093C9048093CA0411
:102310009093CB04C093DD04CC2329F040E051EE30
:1023200060E070E004C040E855E260E070E082EEFA
:1023300095E00E94CA2CCF9108959091CC04492F2A
:102340004F7050E0BA016F5F7F4F292F30E0E4E01B
:1023500035952795EA95E1F76217730759F0FA0169
:10236000E353FB4F808381E0890F8F70907F892B2F
:102370008093CC0408956EE770E082EE95E00E94B1
:1023800059060895A3E1B1E0E8ECF1E10C941E2EAA
:10239000E5E8F5E0712C8191882321F0739428E120
:1023A0007212F9CF66ED71E082EE95E00E946E2A1E
:1023B0004AE050E0672D82EE95E00E946B2B80E0B2
:1023C0000E947E0A0E94590B8E010E5F1F4FC12C86
:1023D000D12C7601C39466246A945C2C0E947628E2
:1023E0004B015C012091840530E0A0E1B7E20E943E
:1023F000942D9B01AC01C701B6010E94B62D20911E
:102400007B0530917C0540917D0550917E05620FE2
:10241000731F841F951F2091BB053091BC0540910F
:10242000BD055091BE05261737074807590718F410
:10243000F801608229C08C2D0E94B20961E070E031
:1024400080E090E00E94A528F80110820E94762882
:10245000681979098A099B09643F714081059105D2
:1024600040F40E94C809F8019081981778F780839A
:10247000EDCF50FE05C05D9841985E9A409A04C029
:102480005D9A419A5E9840982FEFC21AD20AE20AEA
:10249000F20A0F5F1F4F8FEFC816D104E104F10459
:1024A00009F09BCFCE019395FC01D82E7FEF68EC0D
:1024B0002E2F281B271510F051E056C0DE01129672
:1024C00051E02FEF41E03D91321710F0322F01C063
:1024D000452F5F5F5F3F11F0232FF5CF4193242FEE
:1024E00030E0A1E0B0E0AC0FBD1FA20FB31F5C93C2
:1024F000413079F0DE01A20FB31F5C93423049F006
:10250000AFEFBFEFAC0FBD1FA20FB31F6C934E3FD9
:1025100078F6A2E0B0E0AC0FBD1FA20FB31F7C9312
:102520004D3F30F6A3E0B0E0AC0FBD1FA20FB31FCC
:102530006C93BECF452F242F30E0FC01E20FF31F38
:102540006081AFEFB0E0AC0FBD1FA20FB31F2C91A5
:10255000621748F44150DC01A40FB11D2C91208377
:102560006C934111E8CF5F5F571520F3372D3695F7
:1025700020E0231770F4DC01A20FB11D4C91522F03
:10258000530FFC01E50FF11D50815C9340832E5FDA
:10259000F0CFF5E8EF2EF5E0FF2E8C01802F8D199E
:1025A000871598F4F801C1908F014AE050E06C2D36
:1025B00082EE95E00E94342B6CE282EE95E00E9460
:1025C000402AF701C1927F01E9CF82EE95E00E9497
:1025D000482A81E0CD5EDE4FEFE00C943A2E1F9248
:1025E0000F920FB60F9211241F932F933F934F9387
:1025F0005F936F937F938F939F93AF93BF93CF938B
:10260000DF93EF93FF93C0918600D0918700809174
:102610008704909188042091A904211155C09E013E
:10262000281B390B8091BF059091C005A091C10571
:10263000B091C20585FD02C036952795253C49E03D
:102640003407B8F140910A0150E060E070E02CE1FD
:10265000B695A795979587952A95D1F70097A105E7
:10266000B10521F481E090E0A0E0B0E08417950787
:10267000A607B707D8F480910A018F3FB9F040E070
:1026800080910A01481780F4842F90E0880F991FE9
:10269000FC01E757FB4F20813181FC01E55FFE4FD4
:1026A000318320834F5FECCF1092AA0410920A016D
:1026B0000BC02D3B82E0380720F080910A01803169
:1026C000D8F08FEF80930A01D0938804C0938704D9
:1026D000FF91EF91DF91CF91BF91AF919F918F913A
:1026E0007F916F915F914F913F912F911F910F902B
:1026F0000FBE0F901F90189510910A0181E0810F75
:1027000080930A01C9010E94DE08E12FF0E0EE0F7C
:10271000FF1FE757FB4F91838083D6CF83E08093E1
:1027200080008AE9809381008091BF0586FD05C005
:10273000809181008064809381008FEF9FEF909360
:1027400089008093880080916F00806280936F0081
:1027500008950E94300D8091D405843011F41092B8
:10276000D40508956F3018F086958058089589E053
:10277000689F802D11240895A0E0B0E0E2ECF3E121
:102780000C94252EC82F0E948228009138041091A5
:10279000390420913A0430913B046B017C01C01A4A
:1027A000D10AE20AF30A9701860149E8C41643E117
:1027B000D406E104F10410F010923C046093380454
:1027C0007093390480933A0490933B042091A904B8
:1027D0008FEF820F8230D8F5E0913C04EE2309F4AC
:1027E0004EC1E13011F482E0B8C1E03108F034C1EB
:1027F00081E08E0F80933C04F0E0E757FB4FC083ED
:10280000803109F0ACC1EBE8F4E0213029F4A1817A
:10281000A695A695808108C080819181A92FA69553
:10282000A695A69596958795A03148F4B0E090E0DE
:10283000AA0FBB1FA55FBE4F11969C938E9310925B
:10284000AA04329684E0E939F807F9F688C1233002
:1028500009F005C1E0913C04E11104C0CF3009F05A
:102860007EC10DC1E83148F481E08E0F80933C04B5
:10287000F0E0E857FB4FC08372C1E83109F0ECC0CB
:10288000C111EAC040E050E0ABE0CA01B3E0880FFC
:10289000991FBA95E1F7A49F9001A59F300D1124CF
:1028A000F901E757FB4F6081E1817E2F77707595C5
:1028B0006795FC01EE0FFF1FE55FFE4F718360839C
:1028C000F901E657FB4FB081B695B695B695E18113
:1028D000FE2FF295FF0FF07E6F2F6B2BE695E6959E
:1028E000E6957E2F777075956795FC01EE0FFF1FBB
:1028F000E35FFE4F71836083F901E557FB4FB081C1
:10290000B295B695B695B370C181DC2FDD0FDD0FA2
:102910006D2F6B2BC295C695C695C370E281E17091
:10292000EE0FEE0F7E2F7C2B75956795FC01EE0F59
:10293000FF1FE15FFE4F71836083F901E357FB4F97
:10294000B081B695E181FE2FF795FF27F7956F2FA0
:102950006B2BE6957E2F777075956795FC01EE0FD2
:10296000FF1FEF5EFE4F71836083F901E257FB4F5B
:10297000B081B295BF70E181FE2FF295F07F6F2F8D
:102980006B2BE295EF707E2F777075956795FC0144
:10299000EE0FFF1FED5EFE4F71836083F901E1577B
:1029A000FB4FB081BB1FBB27BB1FC181DC2FDD0FDD
:1029B0006D2F6B2BCC1FCC27CC1FE281E370EE0F69
:1029C0007E2F7C2B75956795FC01EE0FFF1FEB5E4C
:1029D000FE4F71836083F901EF56FB4FB081B695CE
:1029E000B695E181FE2FF295FF0FFF0FF07C6F2F60
:1029F0006B2BE695E6957E2F777075956795FC01B4
:102A0000EE0FFF1FE95EFE4F71836083F901EE5602
:102A1000FB4F20812295269527703181E32FEE0F01
:102A2000EE0FEE0F6E2F622B732F729576957770E7
:102A300075956795FC01EE0FFF1FE75EFE4F7183F2
:102A400060834F5F5F4F4230510509F01ECF809188
:102A50009F0483FF1092AA0410923C0480C024308B
:102A600009F07DC060913C0461110BC0C83AB1F41B
:102A7000109275051092740588EA0E94610681E043
:102A80006CC0613019F4C093370404C0623031F473
:102A9000C09336048C2F0E9461065AC0E091360420
:102AA0002E2F30E0220F331F462F50E0C90102962F
:102AB000841795073CF0633268F7FA01EA57FB4F39
:102AC000C083E8CF2D5F3F4F8C2F90E0609174055D
:102AD000709175054217530749F4982F8827862768
:102AE0009727909375058093740532C0681779070E
:102AF00069F580913704813049F5E13118F080E1C2
:102B000080933604F0903604CAE8D4E000E010E088
:102B10000F15D0F4FE013197808190E0982F88271F
:102B20002881822B63E0969587956A95E1F70E944C
:102B3000DE08F801EE0FFF1FE55FFE4F91838083F3
:102B40000F5F1F4F2296E4CF1092AA0410923C040C
:102B500080913C04882319F08F5F80933C04CDB7AB
:102B6000DEB7E8E00C94412EE82FF0E0E654FA4F8F
:102B7000E185E03150F4F894F0E0EE0FFF1FE55FDF
:102B8000FE4F8081918178940895E03121F0E13108
:102B900031F483E101C082E10E94C429089580E0FC
:102BA00092E00895A2E2B0E0E8EDF5E10C941B2E6E
:102BB0009E012F5F3F4F80E1D9011D928A95E9F771
:102BC00064E072E082EE95E029A33AA30E946E2AA7
:102BD0000E947C0B1D8A1E8A1F8A188E312C212C84
:102BE00000E0812C912C540170E4472E71EE572E99
:102BF0007DE9672E78E1772EE0E5CE2EE3ECDE2E40
:102C0000E12CF12C84EF91E0A0E0B0E08D8F9E8F5D
:102C1000AF8FB8A380EC91EDA8E9BBE1898F9A8FC3
:102C2000AB8FBC8F80E491EEADE9B8E1898B9A8BD4
:102C3000AB8BBC8B82EE95E00E94822B892B09F432
:102C4000E1C082EE95E00E94AF2B9C0133272C322D
:102C5000310509F442C0ACF42332310509F0ABC0B0
:102C600019821A821B821C821D821E821F82188674
:102C700019861A861B861C861D861E861F86188A44
:102C800060C02434310529F02335310509F4B2C080
:102C900092C064E482EE95E00E94402A2AE030E08F
:102CA00040E451EE6DE978E182EE95E00E94CE2A93
:102CB0006CE282EE95E00E94402A2AE030E040EC8F
:102CC00051ED68E97BE182EE95E00E94CE2A6CE24C
:102CD00082EE95E00E94802AADCF0F5F043009F0AC
:102CE000A9CF29813A814B815C81A8EEB3E00E9493
:102CF000A32D698B7A8B8B8B9C8B2D813E814F8191
:102D000058850E94A32D698F7A8F8B8F9C8F298580
:102D10003A854B855C852D8F3E8F4F8F58A32D852F
:102D20003E854F8558890E94A32D6B017C0160323E
:102D30003EE473078105910530F462E38CE10E9463
:102D40009F0900E077CF603345E77407810591055F
:102D500010F462E2F3CF60345CE9750781059105F8
:102D600010F466E2EBCF80E5C81683ECD806E104E8
:102D7000F10410F462E1E2CF90E6C9169AEED906AA
:102D8000E104F10410F465E1D9CFA0E7CA16A1E18E
:102D9000DA06A1E0EA06F10410F461E0CFCFB0EA70
:102DA000CB16B6E8DB06B1E0EB06F10410F463E005
:102DB000C5CF65E0C3CF10ED180F1A3008F03ACF39
:102DC000E1E0F0E0EC0FFD1F24E0029FE00DF11DBB
:102DD00011242081318142815381AAE0B0E00E9418
:102DE000A32D610F711D811D911D608371838283ED
:102DF000938320CF49885A886B887C88812C912CBA
:102E0000540118CF81149104A104B10489F4C301C1
:102E1000B2010E940E0A61E070E080E090E00E9442
:102E2000A5281D8A1E8A1F8A188E312C22242A94D6
:102E30008D8D9E8DAF8DB8A188169906AA06BB060A
:102E4000D0F40E94C8092D893E894F89588D280FDA
:102E5000311D411D511D2D8B3E8B4F8B588F3816C8
:102E600008F4382E821508F4282E3FEF831A930AAF
:102E7000A30AB30A56C0C301B20128EE33E040E012
:102E800050E00E94DA2DBA01A9012AE030E082EE7A
:102E900095E00E94252B6CE282EE95E00E94402A8C
:102EA0004AE050E0632D82EE95E00E94342B6CE204
:102EB00082EE95E00E94402A6D897E898F89988DE7
:102EC000A50194010E94DA2DBA01A9012AE030E09F
:102ED00082EE95E00E94252B6CE282EE95E00E9446
:102EE000402A4AE050E0622D82EE95E00E94342BA9
:102EF0006CE282EE95E00E94802A4C0C5D1C6E1CF8
:102F00007F1C898D9A8DAB8DBC8D84159505A6058A
:102F1000B70520F449885A886B887C88812C912CCD
:102F2000540129893A894B895C89283E33404105FF
:102F3000510509F07FCEA296E2E10C94372EACE168
:102F4000B0E0E5EAF7E10C94252E0E9482286B019F
:102F50007C0181E00E947E0A14E703E0198361E0AE
:102F6000CE0101960E94DB0B009373050E94590B62
:102F70006AEF70E080E090E00E94A52880917305E0
:102F8000833089F482EE95E00E94822B892B59F4DC
:102F90000E9482286C197D098E099F096038734C44
:102FA000894C9140D8F280917305833009F44FC069
:102FB0008FE70E9477090E948A098983843511F07E
:102FC00083E05CC00E948A09109246058093470501
:102FD0000E948A092091460530914705280F311D2E
:102FE00030934705209346050E948A09809348053F
:102FF0000E948A0980934905813110F7F12C0F2D29
:1030000010E08091490590E0880F991F0817190773
:1030100040F40E948A09F801E65BFA4F8083F3943A
:10302000EECF80E7898361E0CE0101960E94DB0B41
:1030300083E0809373050E94590B62E370E080E0A7
:1030400090E00E94A52880917305833011F482E0FE
:1030500015C08FE70E9477090E948A09898380350D
:1030600009F0AECF0FE915E00E948A09F8018193BB
:103070008F01F5E00A3B1F07B9F781E06C96E8E0A5
:103080000C94412E80914505992787FD9095A92F95
:10309000B92FFC013196EB30F10508F066C0EC5C0D
:1030A000FF4F0C94522E62E778E082EE95E00E948A
:1030B0005C2A83E893E00E94300C6AE578E082EEB7
:1030C00095E00E945C2A65E378E082EE95E00E943C
:1030D0005C2A6BE078E082EE95E00E945C2A6AEE62
:1030E00077E082EE95E00E945C2A6DEB77E082EE5D
:1030F00095E00E945C2A67E977E082EE95E00E9405
:103100005C2A63E777E082EE95E00E945C2A6CE43B
:1031100077E082EE95E00E945C2A82EE95E00E94C4
:10312000482A0E94700D21C06FE277E01AC06AE061
:1031300077E017C065EF76E014C066ED76E011C069
:1031400062E976E00EC06DE776E00BC068E676E0F7
:1031500082EE95E00E945C2A62E276E002C06CE0BA
:1031600076E082EE95E00E945C2A6AE070E080E002
:1031700090E00E94A52882EE95E00E94822B892B88
:1031800029F082EE95E00E94AF2BF5CF0895ACE1D7
:10319000B0E0EDECF8E10C94252E909145059F3FB1
:1031A00009F023C1482F50E0FA013A97EF36F105B4
:1031B00008F00FC1E15CFF4F0C94522E61E172E008
:1031C000A0C06DE172E082EE95E00E946E2A85E774
:1031D00089838BE1EFE9F5E0DE01129601900D9213
:1031E0008A95E1F76CE1CE0101960E94DB0B0E940B
:1031F000590B83E08093730568EC70E080E090E009
:103200000E94A52880917305843009F0E2C08FE701
:103210000E9477090E948A098983853509F0D9C0FF
:103220006DEE74E082EE95E00E945C2A6FEC74E033
:1032300082EE95E00E945C2A61EB74E096C065E343
:1032400072E082EE95E00E946E2A89E6898361E051
:10325000CE0101960E94DB0B0E94590B83E0809304
:10326000730568EC70E080E090E00E94A5288091F2
:103270007305843009F0ADC08FE70E9477090E9482
:103280008A0989838E010E5F1F4F7E014DE1E40E96
:10329000F11C0E948A09F80181938F01EE15FF0548
:1032A000C1F78BE1FE013296AFE9B5E001900D92D6
:1032B0008A95E1F78981893409F08BC063E974E06C
:1032C00082EE95E00E945C2A65E774E082EE95E06C
:1032D0000E945C2A67E574E048C06FE472E082EE09
:1032E00095E00E946E2A8EEF8093450572C0805251
:1032F0008750805390914805981708F066C06EE596
:1033000072E082EE95E00E946E2A63C084E18093B1
:10331000450560E274E029C085E18093450569EECA
:1033200073E023C086E18093450562EB73E01DC026
:1033300087E18093450568E673E017C088E18093D4
:10334000450567E573E011C089E18093450563E4B5
:1033500073E00BC08AE1809345056EE273E005C01F
:103360008BE18093450566E073E082EE95E00E9474
:103370005C2A2FC06CEE72E082EE95E00E945C2A1F
:103380008091AD0591E01DC066ED72E082EE95E0A2
:103390000E945C2A8091AD0592E013C061EC72E05E
:1033A00082EE95E00E945C2A8091AD0594E009C010
:1033B00066EA72E082EE95E00E945C2A8091AD059B
:1033C00098E089278093AD058FEF809345050E9493
:1033D000111082EE95E00E94822B892B09F45BC1CB
:1033E00082EE95E00E94AF2BF4CF0E94101188234B
:1033F00009F451C18091DF04811104C08FEF8093E3
:10340000450541C140E050E060E070E080EE94E0AE
:103410000E94C92E40914505042F112707FD1095E4
:10342000212F312FF8013197EB31F10508F01BC145
:10343000E255FF4F0C94522E552747FD5095209191
:10344000480530E0241735070CF40DC18B019C01B1
:1034500001501109210931090032110521053105F9
:1034600058F0C0904905EBE4F5E0F12CD12CA8E22E
:10347000EA2E415051090FC0FA01E156FA4F61504E
:103480006083D9C0DF0111972C9130E024173507F4
:1034900029F0F3943296FC10F5CFCBC00E2D10E03E
:1034A00020E030E0061717072807390741F420818C
:1034B000DA01A156BA4F11962C93DD24D394E394EC
:1034C000E8CF6F3F71058105910511F008F0CBC081
:1034D0006093B705B0C06F3F71058105910511F08C
:1034E00008F0C1C06093B805A6C06F3F71058105A3
:1034F000910511F008F0B7C06093B9059CC0209108
:10350000E00420622037E9F440E050E060E070E041
:1035100081EE94E00E94C92E9B01AC01DC01CB013D
:103520000197A109B1090897A105B10508F0AEC03E
:10353000A4EDB0E30E94A32D6A5E7C4A8A46954EB4
:1035400024C02636E9F440E050E060E070E081EE0F
:1035500094E00E94C92E9B01AC01DC01CB010197D4
:10356000A109B1090797A105B10508F08FC0A8EA24
:10357000B1E60E94A32D645E7C438E46944E05C046
:10358000611571058105910579F08B019C0100544D
:10359000114E2D4938410138F0EF1F07FAEF2F0780
:1035A000F2E03F0708F05FC06093AF057093B0058D
:1035B0008093B1059093B2053EC06F3F71058105C0
:1035C000910511F008F04FC06093B30534C08B0132
:1035D0009C0101501109210931090F3F11052105F5
:1035E000310508F040C06093B40525C08B019C01F3
:1035F000045C1940210931090D344DE114072105FE
:10360000310528F47093B6056093B50514C06115B3
:1036100071058105910521F48FEF8093AE050BC0F4
:103620006134710581059105F0F461506093AE0538
:1036300002C0DD20C1F08091DE0481111AC08091AA
:103640007F0590918005A0918105B091820501963A
:10365000A11DB11D80937F0590938005A0938105E6
:10366000B093820506C060E772E082EE95E00E94AA
:103670006E2A0E9406118FEF809345056AE082EE64
:1036800095E00E94802A0E94111005C061E070E060
:1036900080E090E07ACF6C96E8E00C94412E6AE5E9
:1036A00072E082EE95E00E945C2A62E472E082EEB3
:1036B00095E00E945C2A82EE95E00E94822B892B85
:1036C00031F082EE95E00E94AF2B0E94C7180E9455
:1036D0009F17823029F0833051F46DE072E002C010
:1036E00064E272E082EE95E00E945C2A08958FEF1A
:1036F000809345051092DE040E94111080914505CB
:103700008E3F69F082EE95E00E94822B892BB1F307
:1037100082EE95E00E94AF2B0E94C718EFCF08956C
:103720000F931F93109145051F3F09F0D2C08934B4
:1037300009F457C000F5883309F469C058F48033A0
:1037400009F477C008F061C08B3109F440C08132C0
:10375000B1F1B9C0813409F487C030F4893309F478
:1037600066C0803461F1AFC0823409F48EC0863403
:1037700009F448C0A8C0823609F487C078F48835B7
:1037800031F128F48235C1F18335E1F09CC08A35EE
:1037900009F494C0813609F467C095C0823761F19D
:1037A00028F4863679F18936E1F08DC0883779F0D2
:1037B0008A3709F483C0833709F085C003C061E10B
:1037C00072E015C00E94410D6EE872E004C00E94D4
:1037D0004A0D68EA72E082EE95E00E946E2A8EEF52
:1037E00070C00E947A060E94BF0667EC72E082EE0B
:1037F00095E00E946E2A67C081E00E94DF0660EEBD
:1038000072E0F5CF0E94BB105EC080535AC06AEFD1
:1038100071E082EE95E00E945C2A90919E0588E01E
:10382000890F8871977E892B80939E051AC089E045
:1038300048C067EE71E082EE95E00E945C2A8091BC
:10384000BF059091C005A091C105B091C20520E1CE
:1038500082278093BF059093C005A093C105B093C4
:10386000C205109345052FC061ED71E082EE95E031
:103870000E945C2A8091BF059091C005A091C1056E
:10388000B091C20540E4842710C060EC71E082EE84
:1038900095E00E945C2A8091BF059091C005A0919F
:1038A000C105B091C20520E282278093BF059093A5
:1038B000C005A093C105B093C20502C00E944F1B72
:1038C0008FEF80934505809145058E3F09F0D4C068
:1038D000DDC00E941011882309F4D8C08091DF0454
:1038E000811104C08FEF80934505C6C040E050E0D1
:1038F00060E070E080EE94E00E94C92E00914505E2
:10390000112707FD1095212F312FF8013197E9304C
:10391000F10508F0B4C0E753FF4F0C94522E8B0111
:103920009C010154114E2D4938410F37104F2A4F39
:10393000324008F0A4C060937B0570937C058093AF
:103940007D0590937E0577C060937F057093800519
:10395000809381059093820581E08093DE046BC0A3
:10396000683071058105910508F089C06093830571
:1039700062C08B019C0101501109210931090A30F3
:1039800011052105310508F07AC06093840553C004
:1039900061EB71E080EE94E00E94033010E000974C
:1039A00099F00E94DD2F009779F0183130F4E12F63
:1039B000F0E0EA58FA4F87871F5F61EB71E080E023
:1039C00090E00E940330EBCF1831A8F5E12FF0E032
:1039D000EA58FA4F17861F5FF7CF653071058105EA
:1039E000910508F04CC060939D0525C08B019C019A
:1039F0000150110921093109063011052105310550
:103A0000F0F520919E05287F262B20939E0513C05C
:103A10008B019C0101501109210931090115124C3A
:103A20002140310560F560937705709378058093A8
:103A3000790590937A058091DE04811113C08091FD
:103A40007F0590918005A0918105B0918205019636
:103A5000A11DB11D80937F0590938005A0938105E2
:103A6000B09382050E9406118FEF809345056AE0AE
:103A700082EE95E00E94802A0E94421807C060E70B
:103A800072E082EE95E00E946E2AECCF1F910F91BA
:103A900008958FEF809345051092DE040E9442182E
:103AA000809145058E3F69F082EE95E00E94822B61
:103AB000892BB1F382EE95E00E94AF2B0E94901B00
:103AC000EFCF6AE070E080E090E00E94A52882EEEF
:103AD00095E00E94822B892B29F082EE95E00E94CE
:103AE000AF2BF5CF0895CF93C82F682F82EE95E0C6
:103AF0000E94DC2B90916A059C2790936A05CF91D8
:103B00000895A1E0B0E0E7E8FDE10C942B2E998345
:103B10000E94731D9981892F0E94731D2196E2E0F6
:103B20000C94472E1F93CF93DF93182FEB01109225
:103B30006A0565EB70E082EE95E00E94590662E648
:103B400070E082EE95E00E945906812F0E94731D5D
:103B5000CE010E94811DDF91CF911F910895609148
:103B60006A0582EE95E00E94DC2B0895A1E2B0E0A8
:103B7000ECEBFDE10C94272E7B018A018C3009F4DB
:103B800052C108F040C0863009F4BCC018F583303B
:103B900009F491C070F4813009F472C0823009F0E8
:103BA00047C26BE170E082E00E94921D0FE915E0D0
:103BB00078C0843009F487C0853009F039C260913B
:103BC000490570E0660F771F85E00E94921D0AE4A8
:103BD00015E086C0893009F4A7C070F4873009F475
:103BE0009BC0883009F024C261E070E088E00E9448
:103BF000921D8091D40522C28A3009F4CAC08B304C
:103C000009F4F1C015C28A3609F474C1D8F48736B4
:103C100009F439C138F4853609F40DC1863609F442
:103C20001EC106C2883609F436C1893609F000C2C1
:103C300061E070E089E60E94921D0E947A060E946F
:103C4000BF06F4C18D3609F4D3C138F48B3609F4BC
:103C500090C18C3609F499C1EBC18E3609F4DBC1F1
:103C6000873C09F0E5C161E070E087EC0E94921D9D
:103C700081E00E94731D0E94AF1D10926B05E2C18E
:103C800069E270E081E00E94921D06E715E0F8010C
:103C900081918F010E94731DF5E00F391F07B9F75D
:103CA000CFC1F80181918F010E94731DF5E00A3B9D
:103CB0001F07B9F7C5C161E070E083E00E94921D63
:103CC0000E949F17BBC161E070E084E00E94921DDA
:103CD00081E00E94731D0E94AF1D0E94D215B2C1E7
:103CE0008091490590E0880F991F98012A5435402A
:103CF0002817390708F0A4C1F80181918F010E94AB
:103D0000731DEECF62E070E086E00E94921D83E8B2
:103D100093E00E94811D94C161E070E087E00E9401
:103D2000921D809148058AC186E6898361E0CE01B3
:103D300001960E94DB0B0E94590B83E08093730570
:103D400068EC70E080E090E00E94A5288091730507
:103D50008430D9F48FE70E9477090E948A09898309
:103D6000863469F460E270E089E00E94921D10E2FE
:103D70000E948A090E94731D1150D1F761C161E050
:103D800070E089E00E94921D51C161E070E089E01D
:103D900052C169E170E08AE00E94921D1092BA055A
:103DA000209172058091BF059091C005A091C10539
:103DB000B091C205222311F0806801C08F778093F3
:103DC000BF059093C005A093C105B093C2050AEB4F
:103DD00015E0F80181918F010E94731DF5E0033D0C
:103DE0001F07B9F72DC161E270E08BE00E94921DC0
:103DF0008091AA048F3F39F08091AA0491E0980F36
:103E00009093AA0402C08091AA040E94731D10E03E
:103E1000812F0E94B4150E9409090E94811D1F5F15
:103E20001031B1F70DC161E070E08CE00E94921D8D
:103E30008091D30503C161E070E085E60E94921D88
:103E400089E2E816F10409F0F8C0D801E6E7F5E0E8
:103E50008D91819385E0EF39F807D1F7E7C061E0F4
:103E600070E086E60E94921DEBE1EE16F10409F087
:103E7000E4C0D801EFE9F5E08D91819385E0EA3B5C
:103E8000F807D1F7D3C061E070E087E60E94921D89
:103E90000E94410DCBC061E070E088E60E94921D57
:103EA00085E789838BE1EFE9F5E0DE011296019069
:103EB0000D928A95E1F76CE1CE0101960E94DB0B31
:103EC0000E94590B83E08093730560E273E080E009
:103ED00090E00E94A52880917305843009F0ADC060
:103EE0008FE70E9477090E948A098983853509F046
:103EF000A4C09CC061E070E08AE60E94921D89E641
:103F0000898361E0CE0101960E94DB0B0E94590B70
:103F100083E08093730560E273E080E090E00E94AC
:103F2000A52880917305843009F087C08FE70E942F
:103F300077090E948A0989838E010E5F1F4F7E01D7
:103F4000EDE1EE0EF11C0E948A09F80181938F01C8
:103F5000EE15FF05C1F78BE1FE013296AFE9B5E042
:103F600001900D928A95E1F78981893409F065C045
:103F70005DC061E070E08BE60E94921DF8018081D7
:103F80008093D4050E944A0D51C061E070E08CE638
:103F90000E94921DF0E2EF16F10461F487E6898336
:103FA00080E2F801DE01129601900D928A95E1F708
:103FB00061E203C087E4898361E0CE0101960E943B
:103FC000DB0B0E94590B83E0809373056CE474E073
:103FD00080E090E00E94A52880917305843069F507
:103FE0008FE70E9477090E948A09873431F51EC045
:103FF00061E070E08DE60E94921D89E1E816F1040F
:10400000E1F4D801EAEBF5E08D91819385E0E33DA1
:10401000F807D1F70BC061E070E08EE60E94921DB8
:10402000F80180818093D3050E942B0D81E006C0AA
:1040300061E070E08AEC0E94921D80E00E94731D96
:104040000E94AF1DA196E6E00C94432EA0E0B0E0E4
:10405000ECE2F0E20C94252ECAECD3E014E606E084
:1040600035E0F32E44E0E42E53E0D52E62E0C62E78
:1040700082EE95E00E94822B892B09F49BC082EE90
:1040800095E00E94AF2B282F809335044091340493
:1040900050E04730510560F7FA01EE52FF4F0C94A3
:1040A000522E853B29F781E080933404E1CF82369C
:1040B00009F07DC0C0923404DBCF80933304809339
:1040C0003204D0923404D4CF9C013327309331048E
:1040D0002093300490913204982790933204E09218
:1040E0003404C6CF382F2227409130045091310438
:1040F000242B352B309331042093300490913204DB
:10410000982790933204F09234042536310508F450
:10411000AFCF61E070E08CEC0E94921D81E00E94C4
:10412000731D0E94AF1D43C020912E0430912F04B7
:10413000F901E653FC4F80839091320498279093C5
:104140003204C901019690932F0480932E0420918C
:104150003004309131048217930708F489CF00931B
:10416000340486CF8091320482130BC060912E04F8
:1041700070912F044AEC53E0809133040E94B61DE5
:104180000DC062E070E08BEC0E94921D80913304C0
:104190000E94731D80916A050E94731DFE01812F8C
:1041A00011928A95E9F710922F0410922E04109222
:1041B00034045ECFCDB7DEB7E8E00C94412E81E049
:1041C00080936B0580916B05882349F082EE95E022
:1041D0000E94822B892BB1F30E942620F3CF0895F1
:1041E000AAE2B0E0E6EFF0E20C94232E0E947628DB
:1041F0006B017C0181E00E947E0A82EE95E00E94C4
:10420000822B892B29F082EE95E00E94AF2BF5CF0F
:104210005E98409811E072E6B72EE9E2AE2E03E018
:104220000E9476286C197D098E099F09693C7105E9
:1042300081059105E0F11123D1F10E9476286B01EF
:104240007C015D9A419A80ED97E00E94A807B982AF
:10425000E6E7F5E0DE0112968A2D01900D928A952F
:10426000E1F76AE2CE0101960E94DB0B5D9841986E
:1042700080E090E00E94A807009373050E94590B0C
:1042800062E370E080E090E00E94A52880917305D1
:10429000843061F4009373058FE70E9477090E94D0
:1042A0008A0911E0823419F410E001C011E083E1C1
:1042B0000E949B29892BA1F411E012C05E9A409ABA
:1042C0005D9A419A82EE95E00E94AF2B8D30910568
:1042D000B9F06CF40A97A1F05E9840985D98419807
:1042E00082EE95E00E94822B892B41F799CF833291
:1042F000910579F08234910579F70E94DF20ECCFA7
:1043000062EB71E082EE95E00E945C2A0E94491DFA
:10431000E3CF0E94D215E0CF8F929F92AF92BF92CF
:10432000CF92DF92EF92FF921F93CF93DF9383E1BF
:104330000E949B29892B09F089C068EC70E080E01D
:1043400090E00E94A52880E090E00E94A8070E94CB
:1043500076284B015C016B017C0180ECC80E82E188
:10436000D81EE11CF11C0E9476286C157D058E0577
:104370009F0530F483E10E949B29892BA1F364C03F
:1043800083E10E949B29892B09F05EC080ED97E0B4
:104390000E94A8070E9476286B017C01D0E0C1E052
:1043A00088E4880E86E2981EA11CB11C11E083E10E
:1043B0000E949B29892B21F58C149D04AE04BF0417
:1043C00030F480ED97E00E94A807D1E0F0CF0E9482
:1043D00076286C197D098E099F09693C7105810554
:1043E000910528F30E9476286B017C01C12719F002
:1043F00080ED97E002C080E090E00E94A807D7CF50
:1044000080E090E00E94A807DD23B9F08091D305F9
:1044100090E0019665E070E00E94C62D8093D30580
:104420000E942B0D0E94A9130E944A0D64EF71E0B7
:1044300080E090E00E94A52809C080E00E94DF068D
:104440000E94C2110E94410D0E94F020DF91CF9185
:104450001F91FF90EF90DF90CF90BF90AF909F9013
:104460008F900895CF92DF92EF92FF9280E00E94AA
:10447000DA070E94B10761E086E00E942F2961E01F
:1044800085E00E942F2961E08EE00E942F2961E0E3
:104490008FE00E942F2960E083E10E942F2960E0D5
:1044A00088E00E942F2961E088E00E9468290E942C
:1044B0009F0740E052EC61E070E082EE95E00E94E0
:1044C000CA2C0E94A9130E944A0D0E948E138FEFDE
:1044D0008093AA040E94C60778940E9476286B01F4
:1044E0007C018091AA048F3F59F40E9476286C19B0
:1044F0007D098E099F09603D77408105910588F30C
:1045000080ED97E00E94A80761E083E10E9468299E
:104510005E9A409A82EE95E00E94822B892B29F0C8
:1045200082EE95E00E94AF2BF5CF6DEF72E082EE48
:1045300095E00E943D2A83E893E00E94300C64E1FC
:1045400073E082EE95E00E943D2A4AE050E067E089
:1045500070E082EE95E00E940D2B62E370E080E057
:1045600090E00E94A52882EE95E00E94822B04979D
:104570000CF182EE95E00E94AF2B82349105D1F4CC
:1045800082EE95E00E94AF2B8E34910599F482EE75
:1045900095E00E94AF2B8434910561F482EE95E0A2
:1045A0000E94AF2B819731F480E090E00E94A80731
:1045B0000E94F0204091770550917805609179052F
:1045C00070917A05DB01CA010197A109B10904972D
:1045D000A105B10568F44093A904433029F440EAE9
:1045E00056E861E070E004C040E052EC61E070E049
:1045F00082EE95E00E94CA2C0E948C215E98409821
:1046000080E090E00E94A8070E948E131092C504DB
:104610008091BF0583FF11C080918B05882351F0E5
:1046200080919205882331F080919905882311F0BB
:1046300087E001C085E08093C50480E00E947E0A87
:104640008091C6040E94B2090E94590B10923F0447
:1046500010923E0410923D04F12C8091D4058F15E8
:10466000B0F062E370E080E090E00E94A52880ED69
:1046700097E00E94A80762E370E080E090E00E946B
:10468000A52880E090E00E94A807F394E6CF8091EF
:104690009E0584FF08C0982F987181E0983109F039
:1046A00080E00E947E118FE00E94DA07FF90EF9079
:1046B000DF90CF900895EF92FF920F931F93CF93C7
:1046C000DF938C016EE770E082EE95E00E94590660
:1046D000E801F12CF0E2EF2E8E0188818D578230B7
:1046E00048F46DE770E082EE95E00E9459068881FB
:1046F0008E2588832196F801608182EE95E00E94E4
:10470000DC2BF394F9E0FF12E7CF6EE770E082EE66
:1047100095E00E945906CDB7DEB7E6E00C94432E33
:10472000A9E0B0E0E6E9F3E20C942B2E9091C704E7
:1047300091110EC09EEF99838A836B8350E055954B
:1047400047954C832D83198618861F821E822EC0A2
:104750004091CC04842F90E0B4E095958795BA956C
:10476000E1F7242F2F7030E08217930719F18DEFB6
:1047700089831B82FE01349650E0842F90E0A4E0F0
:1047800095958795AA95E1F7242F2F7030E0821731
:10479000930749F0DC01A353BB4F8C918193405F99
:1047A0005F5F563051F74093CC045A83CE01019697
:1047B0000E945B238091C70490E0019666E070E060
:1047C0000E94C62D8093C7042996E2E00C94472EE0
:1047D000A0E0B0E0EEEEF3E20C94242E6C016EE764
:1047E00070E082EE95E00E9459068601E12CF12CE2
:1047F000C0E0D0E030E2B32EF801608183E8860F9C
:10480000823078F46DE770E082EE95E00E94590600
:10481000F80160816B2570E082EE95E00E945906F8
:1048200004C082EE95E00E94DC2BE114F10459F003
:10483000F80180819E01280F311DC901C92FDD2794
:10484000C80FD91FDD273FEFE31AF30A89E0E81606
:10485000F10459F028E0E216F10421F48C2F809540
:10486000F60180870F5F1F4FC7CFCDB7DEB7E9E0F6
:104870000C94402EA9E0B0E0E0E4F4E20C942B2E7E
:10488000E82F362F8091C70490E0019664E270E033
:104890000E94C62D8093C70458E9598350E15A837A
:1048A000813089F048F08230B9F08330D9F48B83BD
:1048B00081EF8C833D8319C085E08B8381EF8C83EE
:1048C0002F5F2D8312C08B8381EF8C8384E6489FFA
:1048D000A00111245D8309C084E08B8381EF8C8368
:1048E000ED8303C00E94BB1104C0CE0101960E945B
:1048F000E8232996E2E00C94472EA2E0B0E0E3E83A
:10490000F4E20C94202E182F762E2A8349830E94DD
:1049100082286B017C018091DD048090C804909016
:10492000C904A090CA04B090CB042A81498188238D
:10493000C1F0D701C60188199909AA09BB094C0120
:104940005D0191EE89169EE29906A104B10420F161
:10495000241708F4422F202F672D812F0E943A241C
:1049600013C0D701C60188199909AA09BB094C01CE
:104970005D0191E3891695E79906A104B10460F001
:10498000672D812F0E949023C092C804D092C90441
:10499000E092CA04F092CB042296EDE00C943C2EF7
:1049A000A2E2B0E0E6EDF4E20C94212E8CE00E944D
:1049B000990981110FC06CE173E082EE95E00E94CD
:1049C0006E2A5E9A409A80E00E947E0A0E94590BED
:1049D0005E98409882EE95E00E94822B892B01F12F
:1049E00082EE95E00E94AF2B9091A904992319F0D3
:1049F0000E94BC13EFCF40913E0450E09A012F5F1C
:104A00003F4F2F71332760913F0470E0261737071F
:104A100009F3FA01E75BFB4F808320933E04DACF72
:104A200080917305843009F086C00E948228611548
:104A300071058105910549F06093B7047093B8043E
:104A40008093B9049093BA040CC081E090E0A0E098
:104A5000B0E08093B7049093B804A093B904B093E6
:104A6000BA048091AD049091AE0481609093AE043D
:104A70008093AD0483E0809373058FE70E947709EC
:104A800009E614E00E948A09F80181938F01F4E09D
:104A900002371F07B9F72091720480916904982F9B
:104AA000922796FF3BC090E4922790937204982F30
:104AB00098739833F1F410E0212F30E0809169046D
:104AC000877090E0821793074CF11F5F20919E053D
:104AD000812F90E0FC01E759FB4F24FF04C0808147
:104AE0000E949D11E9CF608182EE95E00E94DC2B4F
:104AF000E3CF8F7399F480916A048093B604809118
:104B00006B048093B40480916C048093B30480910F
:104B10006F0490E09093AC048093AB0480913D04CB
:104B2000813019F482E080933D0480913D0483300C
:104B300011F410923D040E9482286B017C01809147
:104B4000AF049091B004A091B104B091B204009769
:104B5000A105B105C9F0A7019601281B390B4A0B25
:104B60005B0BDA01C901883B9B40A105B10560F0F0
:104B70000E94C8098093B5041092AF041092B0044B
:104B80001092B1041092B2048091BB049091BC04C5
:104B9000A091BD04B091BE0446015701881A990A3C
:104BA000AA0ABB0A86E795E00E94F40786169706D4
:104BB000A806B90608F4A9C0C092BB04D092BC04F0
:104BC000E092BD04F092BE040E9457068091AA04B0
:104BD0008830A0F08091BF059091C005A091C105DB
:104BE000B091C2055CE1B695A795979587955A95C2
:104BF000D1F7892B8A2B8B2B09F0A2C18091AA04B3
:104C00008F5F8093AA048091B7049091B804A0911B
:104C1000B904B091BA040097A105B105F1F0C81A22
:104C2000D90AEA0AFB0A86E795E00E94F4076C15A8
:104C30007D058E059F0508F008C18091BF0584FDA4
:104C400004C080ED97E00E94A8071092B70410926C
:104C5000B8041092B9041092BA0490917204907C36
:104C60009093720450913E0480913F0420913D0442
:104C7000581709F407C1223009F004C190589093E5
:104C80007204E0919E05E770F0E0E658FC4F608109
:104C9000693008F0DFC0615040E04613DDC080930A
:104CA0003F0487E3840F90917204892B80937204F0
:104CB0004093400483E080933D045D9A419A809143
:104CC00083059091C50491112CC10E94790A8091AD
:104CD000C6040E94B209E0919E05E770F0E0E65834
:104CE000FC4F608182E794E00E94940BE091C6043F
:104CF000EF5FE093C604E83109F41FC1F0E0EA5821
:104D0000FA4F8785882309F418C10E94030C81306B
:104D100069F580919E05887149F18091AD0490916B
:104D2000AE04880F991F9093AE048093AD0483E086
:104D3000809373050E94590B0E9482286093AF04F0
:104D40007093B0048093B1049093B204672B682BE6
:104D5000692B61F481E090E0A0E0B0E08093AF04C3
:104D60009093B004A093B104B093B20480919E05D7
:104D700084FF1FC08091AD049091AE048E7F0E948D
:104D80002A09182F6091AB048091B6040E94B213D7
:104D9000482F612F8091B50449A30E94B21300915E
:104DA000D405282F49A16091B3048091B4040E94D6
:104DB0007D245D9841988091C3048130C1F018F042
:104DC0008230B1F1CBC083E10E949B29892B09F08D
:104DD000C5C081E08093C3040E9476286093BF041D
:104DE0007093C0048093C1049093C204B7C083E160
:104DF0000E949B29892B31F50E947628C090BF0420
:104E0000D090C004E090C104F090C2046C197D09F8
:104E10008E099F09693E73408105910508F49EC083
:104E200082E08093C30480ED97E00E94A80796C0BB
:104E300083E10E949B29892B09F490C080E090E0D7
:104E40000E94A8071092C30489C080E090E00E94ED
:104E5000A80703CF68E020CF851709F420CF4F5F64
:104E6000242F30E090E0F901EE58FB4FDC01A75B06
:104E7000BB4F7C917083F901E05CFB4F708301961E
:104E80008F710BCF2430B1F42091400481E494E081
:104E9000A3E7B4E0FC013E2F381B321718F4319120
:104EA0003D93F9CF87E3820F90917204892B809311
:104EB000720400CF8091C304823059F491609093C2
:104EC00072045E9A409A8E010F5F1F4FF12CB80159
:104ED00011C05E98409880913D04811103C081E02B
:104EE00080933D0480913D04833069F784E0809392
:104EF0003D04E9CF8F2D69A37AA30E94B415F80170
:104F0000819391938F01F39469A17AA1F0E1FF124B
:104F1000F1CF80919E0543E754E087700E947908A5
:104F2000CCCE882309F4D1CE2091C40431E0320FD5
:104F30003093C4042913C9CE0DC01092C604E5CE27
:104F40008091AA04883011F45E9A409A89E0809397
:104F5000AA04DBCE1092C4048150B7CEA296ECE036
:104F60000C943D2E8230E8F4E82FF0E0EE0FFF1FA6
:104F7000EB52FA4F71836083813041F08091690078
:104F80008C7F842B80936900E89A08958091690052
:104F9000440F551F440F551F837F842B8093690056
:104FA000E99A08951F920F920FB60F9211242F9332
:104FB0003F934F935F936F937F938F939F93AF93A1
:104FC000BF93EF93FF938091D5059091D605892BE0
:104FD00029F0E091D505F091D6050995FF91EF9163
:104FE000BF91AF919F918F917F916F915F914F9101
:104FF0003F912F910F900FBE0F901F9018951F9209
:105000000F920FB60F9211242F933F934F935F93FC
:105010006F937F938F939F93AF93BF93EF93FF9380
:105020008091D7059091D805892B29F0E091D7057B
:10503000F091D8050995FF91EF91BF91AF919F91A4
:105040008F917F916F915F914F913F912F910F9031
:105050000FBE0F901F9018951F920F920FB60F92D0
:1050600011242F933F938F939F93AF93BF9380917E
:10507000DA059091DB05A091DC05B091DD0530915A
:10508000D90523E0230F2D3720F40196A11DB11D72
:1050900005C026E8230F0296A11DB11D2093D90556
:1050A0008093DA059093DB05A093DC05B093DD05D2
:1050B0008091DE059091DF05A091E005B091E105BA
:1050C0000196A11DB11D8093DE059093DF05A0938D
:1050D000E005B093E105BF91AF919F918F913F9112
:1050E0002F910F900FBE0F901F9018952FB7F89427
:1050F0006091DA057091DB058091DC059091DD050A
:105100002FBF08953FB7F8948091DE059091DF0599
:10511000A091E005B091E10526B5A89B05C02F3F01
:1051200019F00196A11DB11D3FBF6627782F892F69
:105130009A2F620F711D811D911D42E0660F771F2E
:10514000881F991F4A95D1F70895CF92DF92EF9269
:10515000FF92CF93DF936B017C010E948228EB01C9
:10516000C114D104E104F10479F00E9482286C1B7F
:105170007D0B683E7340A0F381E0C81AD108E108B6
:10518000F108C851DC4FECCFDF91CF91FF90EF9049
:10519000DF90CF900895789484B5826084BD84B503
:1051A000816084BD85B5826085BD85B5816085BD22
:1051B000EEE6F0E0808181608083E1E8F0E010823B
:1051C000808182608083808181608083E0E8F0E07C
:1051D000808181608083E1EBF0E080818460808366
:1051E000E0EBF0E0808181608083EAE7F0E080819D
:1051F00084608083808182608083808181608083FD
:105200008081806880831092C1000895833081F08E
:1052100028F4813099F08230A1F008958630A9F009
:105220008730B9F08430D1F4809180008F7D03C045
:10523000809180008F7780938000089584B58F7768
:1052400002C084B58F7D84BD08958091B0008F77B2
:1052500003C08091B0008F7D8093B0000895CF93FC
:10526000DF9390E0FC01ED50F44F2491FC01E95FE5
:10527000F34F8491882349F190E0880F991FFC0136
:10528000E15DF34FA591B4918B5D934FFC01C59106
:10529000D4919FB7611108C0F8948C912095822316
:1052A0008C93888182230AC0623051F4F8948C91E7
:1052B000322F309583238C938881822B888304C07E
:1052C000F8948C91822B8C939FBFDF91CF9108959E
:1052D000A1E0B0E0EEE6F9E20C94292E282F30E0B0
:1052E000F901E152F44F8491F901ED50F44F14911A
:1052F000F901E95FF34F04910023C9F0882321F0FD
:1053000069830E9406296981E02FF0E0EE0FFF1FFC
:10531000EB5DF34FA591B4919FB7F8948C91611117
:1053200003C01095812301C0812B8C939FBF2196D0
:10533000E4E00C94452ECF93DF93282F30E0F90161
:10534000E152F44F8491F901ED50F44FD491F901F9
:10535000E95FF34FC491CC2391F081110E9406299B
:10536000EC2FF0E0EE0FFF1FE55EF34FA591B49137
:105370002C912D2381E090E021F480E002C080E0B8
:1053800090E0DF91CF9108958E3008F08E508770B5
:1053900020919D0190E4299F90011124822B8093FC
:1053A0007C0080917A00806480937A0080917A00FA
:1053B00086FDFCCF809178002091790090E0922BBF
:1053C0000895A0E0B0E0E7EEF9E20C94252E6C0120
:1053D0007A01EB01E60EF71E00E010E0CE15DF05C6
:1053E00061F06991D601ED91FC910190F081E02D81
:1053F000C6010995080F191FF1CFC801CDB7DEB757
:10540000E8E00C94412E6115710589F0DB010D90E7
:105410000020E9F7AD0141505109461B570BDC0153
:10542000ED91FC910280F381E02D0995089580E0D3
:1054300090E00895EF92FF920F931F93CF93DF9325
:105440008C01FB01C0E0D0E064917F018FEFE81A8E
:10545000F80A662361F0D801ED91FC910190F0818A
:10546000E02DC8010995C80FD91FF701EDCFCE0176
:10547000CDB7DEB7E6E00C94432E0E94032A0895D0
:10548000DC01ED91FC910190F081E02D09950895EA
:105490000F931F93CF93DF93EC016DE00E94402A9E
:1054A0008C016AE0CE010E94402A800F911FDF919B
:1054B000CF911F910F9108950F931F93CF93DF9377
:1054C000EC010E941A2A8C01CE010E94482A800F0A
:1054D000911FDF91CF911F910F9108950F931F930B
:1054E000CF93DF93EC010E94032A8C01CE010E942E
:1054F000482A800F911FDF91CF911F910F9108953E
:105500000F931F93CF93DF93EC010E94402A8C01ED
:10551000CE010E94482A800F911FDF91CF911F91E9
:105520000F910895A1E2B0E0E8E9FAE20C94212E8F
:105530007C01C42EE52FCB01D22E19A221E02D151E
:1055400010F02AE0D22E8E010F5D1F4F8D2C912C72
:10555000A12CB12C6C2D7E2FA50194010E94DA2D77
:105560008C2DD29E80191124015011098A3010F41B
:10557000805D01C0895CF8018083211531054105FA
:10558000510521F0C22EE32FCA01E4CFB801C701B3
:105590000E94032AA196ECE00C943D2EA0E0B0E01E
:1055A000E4EDFAE20C94252EEC016A017B01211551
:1055B000310541F4E881F9810190F081E02D642FFB
:1055C00009951DC02A303105A9F477FF12C06DE29C
:1055D0000E94402A8C0144275527BA014C195D09C5
:1055E0006E097F092AE0CE010E94922A800F911F46
:1055F00006C02AE0B701A601CE010E94922ACDB7CB
:10560000DEB7E8E00C94412E9A01AB01662757FD06
:105610006095762F0E94CE2A08950F931F93CF9303
:10562000DF93EC019A01AB01662757FD6095762F59
:105630000E94CE2A8C01CE010E94482A800F911F21
:10564000DF91CF911F910F9108952115310549F4F4
:10565000DC01ED91FC910190F081E02D642F099522
:1056600008950E94922A08959A01462F50E060E022
:1056700070E00E94252B08959A01AB0160E070E074
:105680000E94252B08950F931F93CF93DF93EC0176
:105690000E94252B8C01CE010E94482A800F911F69
:1056A000DF91CF911F910F9108950F931F93CF9387
:1056B000DF93EC019A01AB0160E070E00E94252BC2
:1056C0008C01CE010E94482A800F911FDF91CF915B
:1056D0001F910F9108950F931F93CF93DF93EC01C8
:1056E0009A01462F50E060E070E00E94252B8C016B
:1056F000CE010E94482A800F911FDF91CF911F9108
:105700000F910895FC0124853585F901E05CFF4F78
:1057100080819181F901EE5BFF4F20813181821BF5
:10572000930B8F7399270895FC0184859585FC015F
:10573000E05CFF4F40815181FC01EE5BFF4F208117
:1057400031814217530741F00190F081E02DE80FBD
:10575000F91F808190E008958FEF9FEF0895FC017D
:1057600084859585FC01E05CFF4F40815181FC01FF
:10577000EE5BFF4F208131814217530779F0A08102
:10578000B181A80FB91F8C91208131812F5F3F4FCC
:105790002F7333273183208390E008958FEF9FEF9D
:1057A0000895FC0181A1882329F0A489B5898C91F1
:1057B00086FFFBCF11A20895CF93DF93FC012685CE
:1057C0003785D901A05CBF4F8D919C9111970196AF
:1057D0008F739927E901CE5BDF4F48815981841788
:1057E0009507D9F30D90BC91A02DA20FB31F6C9318
:1057F000A685B785A05CBF4F11969C938E93A68912
:10580000B7892C9181E090E0078C02C0880F991F26
:105810000A94E2F7282B2C9381E081A30488F58970
:10582000E02D80818064808381E090E0DF91CF91E2
:10583000089508951F920F920FB60F9211242F937F
:105840003F934F938F939F93EF93FF938091C0006B
:1058500082FD1CC04091C600809188069091890607
:1058600001968F73992720918A0630918B068217B3
:10587000930771F0E0918806F0918906E85BF94F93
:105880004083909389068093880602C08091C60069
:10589000FF91EF919F918F914F913F912F910F9099
:1058A0000FBE0F901F90189582EE95E00E94822BFC
:1058B000892B11F00E94192C08951F920F920FB698
:1058C0000F9211242F933F938F939F93EF93FF9306
:1058D00020914406309145068091460690914706F6
:1058E0002817390731F48091C1008F7D8093C10062
:1058F00014C0E0914606F0914706EC5FF94F208115
:10590000809146069091470601968F739927909350
:105910004706809346062093C600FF91EF919F9122
:105920008F913F912F910F900FBE0F901F90189560
:10593000A0E0B0E0EEE9FCE20C94212EFC01138221
:10594000128288EE93E0A0E0B0E084839583A68382
:10595000B7838CEB93E09183808375876487578747
:105960004687318B208B138B028BF58AE48AD78A8A
:10597000C68AB18EA08E938E828E8F85848F888901
:10598000858F8989868F8A89878F8B8980A3ECE0B0
:105990000C943D2ECF92DF92EF92FF92CF93DF9344
:1059A000EC016A017B01411581EE58076105710523
:1059B000F9F0EC89FD8981E090E008A002C0880F31
:1059C000991F0A94E2F7808360E079E08DE390E02C
:1059D000A70196010E94DA2D215031094109510990
:1059E0005695479537952795211580E1380798F00A
:1059F000EC89FD89108260E874E88EE190E0A701EF
:105A000096010E94DA2D215031094109510956951C
:105A1000479537952795E889F9893083EA89FB8985
:105A2000208319A2EE89FF89408181E090E09C01EA
:105A30000C8C02C0220F331F0A94E2F7422B4083E2
:105A4000EE89FF8940819C010D8C02C0220F331F1B
:105A50000A94E2F7422B4083EE89FF8940819C0142
:105A60000E8C02C0220F331F0A94E2F7422B4083B0
:105A7000EE89FF8920810F8C02C0880F991F0A943C
:105A8000E2F7809582238083DF91CF91FF90EF90A2
:105A9000DF90CF9008958F929F92AF92BF92CF9256
:105AA000DF92EF92FF920F931F9381E08F9385E037
:105AB0008F9387E08F9383E08F9384E08F93E6EC5E
:105AC0008E2E912CF2ECAF2EB12CA1ECCA2ED12C43
:105AD000B0ECEB2EF12C04EC10E025EC30E044E0CF
:105AE00056E068E476E082EE95E00E94982C0F90F4
:105AF0000F900F900F900F901F910F91FF90EF90CC
:105B0000DF90CF90BF90AF909F908F9008950E94AC
:105B1000CB280E943222C4E5DCE20E94D0242097E8
:105B2000E1F30E94542CF9CFA29FB001B39FC001B2
:105B3000A39F700D811D1124911DB29F700D811DB9
:105B40001124911D08950E94942DA59F900DB49F3E
:105B5000900DA49F800D911D11240895B7FF0C9402
:105B6000A32D0E94A32D821B930B0895DB018F931D
:105B70009F930E94A32DBF91AF91A29F800D911D75
:105B8000A39F900DB29F900D1124089597FB072EAF
:105B900016F4009407D077FD09D00E94582E07FC18
:105BA00005D03EF4909581959F4F0895709561952D
:105BB0007F4F0895A1E21A2EAA1BBB1BFD010DC049
:105BC000AA1FBB1FEE1FFF1FA217B307E407F507AD
:105BD00020F0A21BB30BE40BF50B661F771F881F89
:105BE000991F1A9469F760957095809590959B011F
:105BF000AC01BD01CF010895052E97FB1EF4009462
:105C00000E94132E57FD07D00E94DA2D07FC03D007
:105C10004EF40C94132E50954095309521953F4F9E
:105C20004F4F5F4F089590958095709561957F4F88
:105C30008F4F9F4F08952F923F924F925F926F9296
:105C40007F928F929F92AF92BF92CF92DF92EF920C
:105C5000FF920F931F93CF93DF93CDB7DEB7CA1B8D
:105C6000DB0B0FB6F894DEBF0FBECDBF09942A88B8
:105C7000398848885F846E847D848C849B84AA8460
:105C8000B984C884DF80EE80FD800C811B81AA81ED
:105C9000B981CE0FD11D0FB6F894DEBF0FBECDBFB8
:105CA000ED010895EE0FFF1F0590F491E02D09948A
:105CB000AA1BBB1B51E107C0AA1FBB1FA617B70732
:105CC00010F0A61BB70B881F991F5A95A9F780954E
:105CD0009095BC01CD0108958F929F92AF92BF9293
:105CE000CF92DF92EF92FF92CF93DF93EC01688126
:105CF00079818A819B81611571058105910521F466
:105D000064E279ED8BE597E02DE133EF41E050E07F
:105D10000E94FC2D49015A019B01AC01A7EAB1E4A4
:105D20000E94A32D6B017C01ACEEB4EFA5019401A0
:105D30000E94B12DC60ED71EE81EF91EF7FE06C042
:105D400081E0C81AD108E10880E8F80AC882D9823F
:105D5000EA82FB82C701B6019F77DF91CF91FF9066
:105D6000EF90DF90CF90BF90AF909F908F9008956D
:105D70000E946C2E089586E091E00E946C2E08959A
:105D800060930601709307018093080190930901C5
:105D900008952F923F925F926F927F928F929F927F
:105DA000AF92BF92CF92DF92EF92FF920F931F9329
:105DB000CF93DF938B01EA016115710521F0DB01BF
:105DC0008C9311969C93209739F09E0122503109B3
:105DD0002332310508F0D8C07C016701BFEFCB1A30
:105DE000DB0A5601F7016080862D90E00E94FB2FB0
:105DF000892B11F07601F1CFFDE26F120AC0570135
:105E000082E0A80EB11CD70111966C907724739490
:105E10000BC0BBE26B1207C05701E2E0AE0EB11C33
:105E2000D70111966C90712CCE018F7E892B89F44D
:105E3000B0E36B1237C0F50180818F7D8835D1F4D6
:105E40006180F2E0AF0EB11C872D8260782EC0E138
:105E5000D0E0CA30D10551F1C031D10521F0C830B0
:105E6000D10599F409C0CC24CA94DC2CEC2CAFE009
:105E7000FA2E22C0209769F7C8E0D0E0CC24CA945B
:105E8000DC2CEC2CFFE1FF2E17C06FEF7FEFCB0176
:105E90009E01442737FD4095542F0E94DA2D690159
:105EA0007A010AC02097A9F6CAE0D0E0E9E9CE2E2F
:105EB000DC2CEC2CE9E1FE2EF50160E020E030E086
:105EC000A9014E01AA2497FCA094BA2C1F0170EDE1
:105ED000572E560CA9E0A51570F48FEB860D8A316C
:105EE00018F499EC592E06C08FE9860D8A3148F5D1
:105EF00089EA582E560C852D90E08C179D070CF5DD
:105F00006F3FD9F0C216D306E406F50698F0C50136
:105F1000B4010E94B62D9B01AC01852D90E0A0E05C
:105F2000B0E0280F391F4A1F5B1F281739074A079F
:105F30005B0710F46FEF01C061E03196D1016C9006
:105F4000C5CF0115110551F0662311F0319703C03B
:105F500071FE04C03297D801ED93FC9370FE07C028
:105F600050954095309521953F4F4F4F5F4F67FFBC
:105F700010C082E290E090938D0680938C066FEFC4
:105F80007FEF8FEF9FEF07C060E070E080E090E070
:105F900002C0B901CA01DF91CF911F910F91FF900B
:105FA000EF90DF90CF90BF90AF909F908F907F90B9
:105FB0006F905F903F902F900895FC01882799275C
:105FC000E89421912032E9F3293010F02E30C8F303
:105FD0002B3241F02D3239F4689404C00E942F30E6
:105FE000820F911D219120532A30C0F31EF4909509
:105FF00081959F4F0895911150C0803219F08950BA
:106000008550D0F7089548EC53E00E940830089579
:10601000FA01A191B081009719F41097E1F0CD0138
:10602000DC01CD010D90002011F4C00113C0FB0173
:106030002191222319F02015D9F7F3CFFB012191EB
:10604000201519F41E92119606C02223C1F70D9057
:106050000020A1F7D001FA01A193B08308957AE05E
:10606000979F902D879F802D910D11240895F99968
:10607000FECF92BD81BDF89A992780B50895262F4D
:10608000F999FECF1FBA92BD81BD20BD0FB6F8941D
:10609000FA9AF99A0FBE01960895992788270895CC
:0460A000F894FFCFA2
:1060A40000008E06200001000000FF000200020034
:1060B40002000200020002000200020002000200CC
:1060C4000200020002000200020002802500000516
:1060D400400AA1204EA50020244EA52C2330C01236
:1060E40000001A400AA1204EA5001B1E27522C2393
:1060F400308025000005400AA1204EA50020244E32
:10610400A52C2330004B000006400AD0009D490016
:106114007B289D492C233000E1000005400A4501FD
:10612400D7DC03B81E0EBF00232E48E801008A40C6
:106134000A6001555502AD1E20000023C8015458C1
:106144002074696D656F75742100596573004E6F15
:10615400002C00386368004E2F41002C205B005D4A
:106164002028002900486F70206368616E6E656C9A
:10617400200020402000456E746572696E672061BE
:1061840064617074697665206368616E6E656C2005
:1061940073656C656374696F6E2C207069636B69D9
:1061A4006E673A007363616E6E6572206D6F64652D
:1061B400004E4F5420454E41424C45440053656EB9
:1061C40064696E672073657474696E677320746F95
:1061D4002052580A00526573657474696E6720739F
:1061E400657474696E6773206F6E2052580A00419B
:1061F400626F727465642065646974730A00696E01
:1062040076616C69642073656C656374696F6E0094
:106214000D0A496E76616C696420696E707574202C
:106224002D2064697363617264656421070053659A
:106234007474696E677320736176656420746F206B
:10624400454550524F4D0A00526576657274656437
:106254002073657474696E67732066726F6D204570
:106264004550524F4D0A004C6F616465642066616D
:1062740063746F72792064656661756C74730A0067
:106284004B657920616E64206368616E6E656C7322
:106294002072616E646F6D697A65640A004F70657F
:1062A4006E4C52536E672054582073746172746933
:1062B4006E672000206F6E20485720006D6F647554
:1062C4006C65206C6F636B65643F00342B3400385D
:1062D40000382B340031320031322B340031360097
:1062E40050504D0052535349005344410053434CC2
:1062F40000525844005458440041494E004C424511
:1063040045500053504B54524D0053425553005383
:10631400554D44004C4C494E440000070B0C1011E1
:106324001500B7012B032F033103350338033D0355
:10633400B7014003440349034D0351035503590373
:106344005D0363036A036F0374038D028D028D0280
:106354008D02160A1322312900000000DC2BE129EA
:08636400822BAF2B942BD12BEF
:00000001FF
